:100000007FC0A7C0A6C0A5C0A4C0B1C0A2C0A1C0E7
:10001000A0C09FC09EC09DC09CC09BC09AC074459C
:1000200079467D47824887498B60906194629963E5
:100030009D64A265A766AB67B068B469B980BE81EC
:10004000C282C783CB84D084D484FF2103030405F8
:1000500006080A0C0F13171C21282F373F49545F3D
:100060006C7A8999ABBED2E8FFFFFFFFFFFFFFFF6D
:10007000FFFFFFFFFFFFFFFFFFFFFFFFFFFFFFFF90
:10008000FFFFFFFFFFFFFFFFFFFFFF00000000007B
:100090000000000000000000000000000000000060
:1000A0000000000000000000000205080B0E121600
:1000B0001A1E22272C31363B41474D545B62697131
:1000C000798189929BA4AEB8C2CDD8FF40000B4085
:1000D000000B2340000B1A2E40000B172432400067
:1000E0000B141F293540001D40F200F3F40B1D4096
:1000F0000009121D2E40000B1D3200F3F4F24000E7
:1001000011241FBECFE5D1E0DEBFCDBF20E0A0E6C9
:10011000B0E001C01D92A338B207E1F7E1E6F0E0DC
:1001200085E5808781E08383148212828683118231
:10013000ACE6B0E08EEF15968C9315978DEF179681
:100140008C9385E081878FE48287612C712CB4D0F9
:10015000A8C256CF815090E0FC01E45BFF4FE491D0
:10016000E9BDFC01E457FF4F849188BD08951895BF
:1001700025B7277E25BF29B7226029BF21E022BFEE
:10018000019728F020E188952150E9F7F9CF0895EB
:1001900088EE93E0EDCF81EA87B986EC86B9369A8E
:1001A0000895369A3699FECF85B10895CF93C72D1D
:1001B00081E0870D8F73782E662D90E064D26FEF0B
:1001C0008C2F90E0CF915FC2FF920F931F93CF933C
:1001D000DF93F82E0BE610E0C5E7D0E081E0F812DF
:1001E00005C0F8016081CE014ED204C0CE0143D2D9
:1001F000F8018083015011092196CF37D10571F79D
:10020000DF91CF911F910F91FF900895CFDF81E093
:10021000DBCF811103C019BC18BC08959BCF0F938D
:100220001F93CF93C82F8B01CC2361F081E192DF24
:10023000C8019EDF19BC18BCC8019ADFC80198DF4D
:10024000C150F2CFCF911F910F910895EF92FF927D
:100250000F931F93CF93C8E0E82EF12C062F10E0E8
:1002600080E478DFC70184DF19BC18BCC80180DFD7
:10027000C150B1F7CF911F910F91FF90EF9008956A
:100280001F93CF93DF938FEA87B986EC86B910E18D
:10029000C0E0D0E085E090E06BDF83DFC80FD11DC8
:1002A0001150C1F7CE0124E0969587952A95E1F784
:1002B000DF91CF911F91089583EA87B986EC86B9C3
:1002C0003699FECF369A3699FECFC5B18FE384BBFF
:1002D000BB9AC39AB99AB89A81E08ABD83BF8AB59E
:1002E00080628ABD8AB580688ABD97B328B3892F9A
:1002F00090E0809590958B7F822B88BB85B780623C
:1003000085BF789487E790E0B6D1853511F07EDF20
:1003100011C0712C872D90E0AED1682E8F3F19F05F
:1003200080E052DF07C0872D91E0970D792E803451
:1003300088F3F6CF80916A0000916400F090650028
:1003400010916200112319F0F12C00E089E08F5F19
:1003500090E040E050E06CEC70E0882379F09B0185
:100360002F5F3F4FF9013197E491EE2319F0922F5F
:10037000961BF6CF8150AB01B901EFCF892F602FCB
:1003800070E0A92FB0E0E82FF0E0FF2021F09D0100
:100390002E1B3F0B05C09F0121503109260F371F2F
:1003A0003197E40FF51FE4902B583F4FF901E0829D
:1003B000815049F7900F90936000002371F0FF2067
:1003C00029F0292F30E02150310902C020E030E02F
:1003D000F901EB58FF4F81E0808384E0890F282FDB
:1003E0002150E22FE91BF0E0E550FF4FE491A22FEE
:1003F000B0E0AB58BF4FEC932913F2CFE82FF0E0F9
:10040000EC58FF4F21E0409175003081431320E00C
:10041000821B282F80938200862D853F70F5C93F6F
:1004200060F08F5F682E891708F0612C809183003F
:100430008F5F8F718093830020C010928300C33D33
:10044000B0F030916700332311F0112331F08F5F4A
:10045000682E891790F0612C10C06916E1F36620B0
:1004600019F08150682E09C02150622E06C011116A
:10047000F2CF80916300882371F398DE8CDEC62D65
:10048000C53F28F4D0E0CB58DF4FC881DC2F10E007
:1004900000E0EE24E39480918300803190F178DED7
:1004A00010928300C2E6D0E0C12CD12C81E08C0DEB
:1004B000FFEFCF1ADF0A98819F3F31F4219688E041
:1004C000C816D10499F718C06DE570E0A8DEF601F2
:1004D000E459FF4F608088818E25888397DE6FE026
:1004E00070E080E29CDE88818E2588838FDE50DE7E
:1004F00080916200882311F3612CC0917500DC2F7C
:100500008DC0C23F39F468E284E1A0DE60E588E294
:100510009DDE84C0C33F91F484E0F82E80E41ADEAF
:1005200085E090E025DE8DE115DE81E490E020DEBF
:10053000FA94F110F3CF80ED92E06FC0C43F59F50B
:1005400084E690E015DE27DE2CDE90E0292F30E0F7
:10055000F901E25EFF4FE491E81710F49E5FF6CFD9
:10056000F901E15EFF4FF4906DE770E08F2D829509
:100570008695877054DE8EEE92E0FADD65E070E0DD
:1005800081E04DDE85E694E0F3DD6DE770E08F2DD0
:100590008F7145DE0FC0CE3F81F4612CF12CF092BB
:1005A0006A0034DE6AEF70E081E039DEF39499E0AE
:1005B000F912F5CFEDDDECDD31C0CD3F91F4612CCA
:1005C0008FEF80936B0022DE80E1C4DDE1DDE0DDB2
:1005D00080E4C0DD55DE80936B0018DED9DDD8DD08
:1005E000F9CF8D2F16DE4CDE20916B00821738F08C
:1005F0000F5F093078F0D93068F0D1500AC090E030
:1006000030E022503109821793071CF4DC1708F4FC
:10061000DF5F00E0C0DD84EF91E0AADD109283008F
:10062000C0DD823890F41F5F183008F434CFD13425
:1006300020F010E0D0E2C0E22ECFD23040F08D2F7B
:1006400086958695D695D80FCD2F10E024CF19BC6E
:1006500018BC85B7877E806185BFF89485B78468AC
:1006600085BF8B7F85BF85B7806285BF889585B73D
:100670008F7D85BFE9CFE199FECF1FBA8EBBE09A8F
:1006800099278DB30895262FE199FECF1CBA1FBA82
:100690008EBB2DBB0FB6F894E29AE19A0FBE01967D
:0606A0000895F894FFCF5D
:00000001FF
